
C:\Documents and Settings\jarek\Pulpit\Privet\Magisterka\Programy\1\um0427\FWLib\project\RIDE\STM3210E-EVAL\SCROLL_M.o:     file format elf32-littlearm
C:\Documents and Settings\jarek\Pulpit\Privet\Magisterka\Programy\1\um0427\FWLib\project\RIDE\STM3210E-EVAL\SCROLL_M.o

Disassembly of section .text.Init:

00000000 <Init>:
Init():
C:\Documents and Settings\jarek\Pulpit\Privet\Magisterka\Programy\1\um0427\FWLib\project/SCROLL_M.c:104
   0:	4b01      	ldr	r3, [pc, #4]	(8 <Init+0x8>)
   2:	2201      	movs	r2, #1
   4:	701a      	strb	r2, [r3, #0]
C:\Documents and Settings\jarek\Pulpit\Privet\Magisterka\Programy\1\um0427\FWLib\project/SCROLL_M.c:105
   6:	4770      	bx	lr
   8:	00000000 	.word	0x00000000
Disassembly of section .text.printFrame:

00000000 <printFrame>:
printFrame():
C:\Documents and Settings\jarek\Pulpit\Privet\Magisterka\Programy\1\um0427\FWLib\project/SCROLL_M.c:82
   0:	b513      	push	{r0, r1, r4, lr}
C:\Documents and Settings\jarek\Pulpit\Privet\Magisterka\Programy\1\um0427\FWLib\project/SCROLL_M.c:84
   2:	f7ff fffe 	bl	0 <GRAPH_ClearScreen>
C:\Documents and Settings\jarek\Pulpit\Privet\Magisterka\Programy\1\um0427\FWLib\project/SCROLL_M.c:85
   6:	f7ff fffe 	bl	0 <GRAPH_WhiteBlack>
C:\Documents and Settings\jarek\Pulpit\Privet\Magisterka\Programy\1\um0427\FWLib\project/SCROLL_M.c:87
   a:	2000      	movs	r0, #0
   c:	2401      	movs	r4, #1
   e:	22ef      	movs	r2, #239
  10:	2314      	movs	r3, #20
  12:	4601      	mov	r1, r0
  14:	9400      	str	r4, [sp, #0]
  16:	f7ff fffe 	bl	0 <GRAPH_Rectangle>
C:\Documents and Settings\jarek\Pulpit\Privet\Magisterka\Programy\1\um0427\FWLib\project/SCROLL_M.c:88
  1a:	2002      	movs	r0, #2
  1c:	22eb      	movs	r2, #235
  1e:	2310      	movs	r3, #16
  20:	4601      	mov	r1, r0
  22:	9400      	str	r4, [sp, #0]
  24:	f7ff fffe 	bl	0 <GRAPH_Rectangle>
C:\Documents and Settings\jarek\Pulpit\Privet\Magisterka\Programy\1\um0427\FWLib\project/SCROLL_M.c:89
  28:	2113      	movs	r1, #19
  2a:	2203      	movs	r2, #3
  2c:	236c      	movs	r3, #108
  2e:	2000      	movs	r0, #0
  30:	9400      	str	r4, [sp, #0]
  32:	f7ff fffe 	bl	0 <GRAPH_Rectangle>
C:\Documents and Settings\jarek\Pulpit\Privet\Magisterka\Programy\1\um0427\FWLib\project/SCROLL_M.c:90
  36:	217d      	movs	r1, #125
  38:	22ef      	movs	r2, #239
  3a:	2303      	movs	r3, #3
  3c:	2000      	movs	r0, #0
  3e:	9400      	str	r4, [sp, #0]
  40:	f7ff fffe 	bl	0 <GRAPH_Rectangle>
C:\Documents and Settings\jarek\Pulpit\Privet\Magisterka\Programy\1\um0427\FWLib\project/SCROLL_M.c:93
  44:	236c      	movs	r3, #108
  46:	2113      	movs	r1, #19
  48:	2203      	movs	r2, #3
  4a:	20ec      	movs	r0, #236
  4c:	9400      	str	r4, [sp, #0]
  4e:	f7ff fffe 	bl	0 <GRAPH_Rectangle>
C:\Documents and Settings\jarek\Pulpit\Privet\Magisterka\Programy\1\um0427\FWLib\project/SCROLL_M.c:96
  52:	217d      	movs	r1, #125
  54:	2200      	movs	r2, #0
  56:	4620      	mov	r0, r4
  58:	f7ff fffe 	bl	0 <GRAPH_SetPixel>
C:\Documents and Settings\jarek\Pulpit\Privet\Magisterka\Programy\1\um0427\FWLib\project/SCROLL_M.c:97
  5c:	2200      	movs	r2, #0
  5e:	4620      	mov	r0, r4
  60:	217e      	movs	r1, #126
  62:	f7ff fffe 	bl	0 <GRAPH_SetPixel>
C:\Documents and Settings\jarek\Pulpit\Privet\Magisterka\Programy\1\um0427\FWLib\project/SCROLL_M.c:98
  66:	2002      	movs	r0, #2
  68:	217e      	movs	r1, #126
  6a:	2200      	movs	r2, #0
  6c:	f7ff fffe 	bl	0 <GRAPH_SetPixel>
C:\Documents and Settings\jarek\Pulpit\Privet\Magisterka\Programy\1\um0427\FWLib\project/SCROLL_M.c:99
  70:	217d      	movs	r1, #125
  72:	2200      	movs	r2, #0
  74:	20ed      	movs	r0, #237
  76:	f7ff fffe 	bl	0 <GRAPH_SetPixel>
C:\Documents and Settings\jarek\Pulpit\Privet\Magisterka\Programy\1\um0427\FWLib\project/SCROLL_M.c:100
  7a:	2300      	movs	r3, #0
  7c:	217e      	movs	r1, #126
  7e:	9300      	str	r3, [sp, #0]
  80:	20e6      	movs	r0, #230
  82:	22ed      	movs	r2, #237
  84:	460b      	mov	r3, r1
  86:	f7ff fffe 	bl	0 <GRAPH_Line>
C:\Documents and Settings\jarek\Pulpit\Privet\Magisterka\Programy\1\um0427\FWLib\project/SCROLL_M.c:101
  8a:	bd1c      	pop	{r2, r3, r4, pc}
Disassembly of section .text.GoBack:

00000000 <GoBack>:
GoBack():
C:\Documents and Settings\jarek\Pulpit\Privet\Magisterka\Programy\1\um0427\FWLib\project/SCROLL_M.c:28
   0:	b573      	push	{r0, r1, r4, r5, r6, lr}
C:\Documents and Settings\jarek\Pulpit\Privet\Magisterka\Programy\1\um0427\FWLib\project/SCROLL_M.c:30
   2:	f7ff fffe 	bl	0 <GRAPH_ClearScreen>
C:\Documents and Settings\jarek\Pulpit\Privet\Magisterka\Programy\1\um0427\FWLib\project/SCROLL_M.c:33
   6:	2000      	movs	r0, #0
   8:	2401      	movs	r4, #1
   a:	22ef      	movs	r2, #239
   c:	2314      	movs	r3, #20
   e:	4601      	mov	r1, r0
  10:	9400      	str	r4, [sp, #0]
  12:	f7ff fffe 	bl	0 <GRAPH_Rectangle>
C:\Documents and Settings\jarek\Pulpit\Privet\Magisterka\Programy\1\um0427\FWLib\project/SCROLL_M.c:34
  16:	2002      	movs	r0, #2
  18:	22eb      	movs	r2, #235
  1a:	2310      	movs	r3, #16
  1c:	4601      	mov	r1, r0
  1e:	9400      	str	r4, [sp, #0]
  20:	f7ff fffe 	bl	0 <GRAPH_Rectangle>
C:\Documents and Settings\jarek\Pulpit\Privet\Magisterka\Programy\1\um0427\FWLib\project/SCROLL_M.c:35
  24:	2113      	movs	r1, #19
  26:	2203      	movs	r2, #3
  28:	236c      	movs	r3, #108
  2a:	2000      	movs	r0, #0
  2c:	9400      	str	r4, [sp, #0]
  2e:	f7ff fffe 	bl	0 <GRAPH_Rectangle>
C:\Documents and Settings\jarek\Pulpit\Privet\Magisterka\Programy\1\um0427\FWLib\project/SCROLL_M.c:36
  32:	217d      	movs	r1, #125
  34:	22ef      	movs	r2, #239
  36:	2303      	movs	r3, #3
  38:	2000      	movs	r0, #0
  3a:	9400      	str	r4, [sp, #0]
  3c:	f7ff fffe 	bl	0 <GRAPH_Rectangle>
C:\Documents and Settings\jarek\Pulpit\Privet\Magisterka\Programy\1\um0427\FWLib\project/SCROLL_M.c:39
  40:	236c      	movs	r3, #108
  42:	2113      	movs	r1, #19
  44:	2203      	movs	r2, #3
  46:	20ec      	movs	r0, #236
  48:	9400      	str	r4, [sp, #0]
  4a:	f7ff fffe 	bl	0 <GRAPH_Rectangle>
C:\Documents and Settings\jarek\Pulpit\Privet\Magisterka\Programy\1\um0427\FWLib\project/SCROLL_M.c:42
  4e:	217d      	movs	r1, #125
  50:	2200      	movs	r2, #0
  52:	4620      	mov	r0, r4
  54:	f7ff fffe 	bl	0 <GRAPH_SetPixel>
C:\Documents and Settings\jarek\Pulpit\Privet\Magisterka\Programy\1\um0427\FWLib\project/SCROLL_M.c:43
  58:	217e      	movs	r1, #126
  5a:	4620      	mov	r0, r4
  5c:	2200      	movs	r2, #0
  5e:	f7ff fffe 	bl	0 <GRAPH_SetPixel>
C:\Documents and Settings\jarek\Pulpit\Privet\Magisterka\Programy\1\um0427\FWLib\project/SCROLL_M.c:44
  62:	217e      	movs	r1, #126
  64:	2002      	movs	r0, #2
  66:	2200      	movs	r2, #0
  68:	f7ff fffe 	bl	0 <GRAPH_SetPixel>
C:\Documents and Settings\jarek\Pulpit\Privet\Magisterka\Programy\1\um0427\FWLib\project/SCROLL_M.c:45
  6c:	217d      	movs	r1, #125
  6e:	2200      	movs	r2, #0
  70:	20ed      	movs	r0, #237
  72:	f7ff fffe 	bl	0 <GRAPH_SetPixel>
C:\Documents and Settings\jarek\Pulpit\Privet\Magisterka\Programy\1\um0427\FWLib\project/SCROLL_M.c:46
  76:	217e      	movs	r1, #126
  78:	2500      	movs	r5, #0
  7a:	22ed      	movs	r2, #237
  7c:	460b      	mov	r3, r1
  7e:	20e6      	movs	r0, #230
  80:	9500      	str	r5, [sp, #0]
  82:	f7ff fffe 	bl	0 <GRAPH_Line>
C:\Documents and Settings\jarek\Pulpit\Privet\Magisterka\Programy\1\um0427\FWLib\project/SCROLL_M.c:48
  86:	4a27      	ldr	r2, [pc, #156]	(124 <GoBack+0x124>)
C:\Documents and Settings\jarek\Pulpit\Privet\Magisterka\Programy\1\um0427\FWLib\project/SCROLL_M.c:55
  88:	4621      	mov	r1, r4
C:\Documents and Settings\jarek\Pulpit\Privet\Magisterka\Programy\1\um0427\FWLib\project/SCROLL_M.c:48
  8a:	6c93      	ldr	r3, [r2, #72]
C:\Documents and Settings\jarek\Pulpit\Privet\Magisterka\Programy\1\um0427\FWLib\project/SCROLL_M.c:55
  8c:	2002      	movs	r0, #2
C:\Documents and Settings\jarek\Pulpit\Privet\Magisterka\Programy\1\um0427\FWLib\project/SCROLL_M.c:48
  8e:	6453      	str	r3, [r2, #68]
C:\Documents and Settings\jarek\Pulpit\Privet\Magisterka\Programy\1\um0427\FWLib\project/SCROLL_M.c:49
  90:	6cd3      	ldr	r3, [r2, #76]
  92:	6493      	str	r3, [r2, #72]
C:\Documents and Settings\jarek\Pulpit\Privet\Magisterka\Programy\1\um0427\FWLib\project/SCROLL_M.c:50
  94:	6d13      	ldr	r3, [r2, #80]
  96:	64d3      	str	r3, [r2, #76]
C:\Documents and Settings\jarek\Pulpit\Privet\Magisterka\Programy\1\um0427\FWLib\project/SCROLL_M.c:51
  98:	6d53      	ldr	r3, [r2, #84]
C:\Documents and Settings\jarek\Pulpit\Privet\Magisterka\Programy\1\um0427\FWLib\project/SCROLL_M.c:52
  9a:	6555      	str	r5, [r2, #84]
C:\Documents and Settings\jarek\Pulpit\Privet\Magisterka\Programy\1\um0427\FWLib\project/SCROLL_M.c:51
  9c:	6513      	str	r3, [r2, #80]
C:\Documents and Settings\jarek\Pulpit\Privet\Magisterka\Programy\1\um0427\FWLib\project/SCROLL_M.c:53
  9e:	6d93      	ldr	r3, [r2, #88]
  a0:	3b01      	subs	r3, #1
  a2:	6593      	str	r3, [r2, #88]
C:\Documents and Settings\jarek\Pulpit\Privet\Magisterka\Programy\1\um0427\FWLib\project/SCROLL_M.c:55
  a4:	f7ff fffe 	bl	0 <GRAPH_TextGoTo>
C:\Documents and Settings\jarek\Pulpit\Privet\Magisterka\Programy\1\um0427\FWLib\project/SCROLL_M.c:56
  a8:	f7ff fffe 	bl	0 <GRAPH_WhiteBlack>
C:\Documents and Settings\jarek\Pulpit\Privet\Magisterka\Programy\1\um0427\FWLib\project/SCROLL_M.c:57
  ac:	481e      	ldr	r0, [pc, #120]	(7c <printf+0x7c>)
  ae:	f7ff fffe 	bl	0 <printf>
C:\Documents and Settings\jarek\Pulpit\Privet\Magisterka\Programy\1\um0427\FWLib\project/SCROLL_M.c:58
  b2:	2002      	movs	r0, #2
  b4:	4621      	mov	r1, r4
  b6:	f7ff fffe 	bl	0 <GRAPH_TextGoTo>
C:\Documents and Settings\jarek\Pulpit\Privet\Magisterka\Programy\1\um0427\FWLib\project/SCROLL_M.c:59
  ba:	e007      	b.n	cc <GoBack+0xcc>
C:\Documents and Settings\jarek\Pulpit\Privet\Magisterka\Programy\1\um0427\FWLib\project/SCROLL_M.c:60
  bc:	f852 0025 	ldr.w	r0, [r2, r5, lsl #2]
  c0:	f7ff fffe 	bl	0 <printf>
C:\Documents and Settings\jarek\Pulpit\Privet\Magisterka\Programy\1\um0427\FWLib\project/SCROLL_M.c:61
  c4:	4819      	ldr	r0, [pc, #100]	(68 <printf+0x68>)
  c6:	f7ff fffe 	bl	0 <printf>
C:\Documents and Settings\jarek\Pulpit\Privet\Magisterka\Programy\1\um0427\FWLib\project/SCROLL_M.c:59
  ca:	3501      	adds	r5, #1
  cc:	4a15      	ldr	r2, [pc, #84]	(124 <GoBack+0x124>)
  ce:	6d93      	ldr	r3, [r2, #88]
  d0:	429d      	cmp	r5, r3
  d2:	ddf3      	ble.n	bc <GoBack+0xbc>
  d4:	4616      	mov	r6, r2
  d6:	2500      	movs	r5, #0
  d8:	e01e      	b.n	118 <GoBack+0x118>
C:\Documents and Settings\jarek\Pulpit\Privet\Magisterka\Programy\1\um0427\FWLib\project/SCROLL_M.c:66
  da:	6c53      	ldr	r3, [r2, #68]
  dc:	42ab      	cmp	r3, r5
  de:	d102      	bne.n	e6 <GoBack+0xe6>
C:\Documents and Settings\jarek\Pulpit\Privet\Magisterka\Programy\1\um0427\FWLib\project/SCROLL_M.c:67
  e0:	f7ff fffe 	bl	0 <GRAPH_BlackWhite>
  e4:	e001      	b.n	6 <GRAPH_WhiteBlack+0x6>
C:\Documents and Settings\jarek\Pulpit\Privet\Magisterka\Programy\1\um0427\FWLib\project/SCROLL_M.c:69
  e6:	f7ff fffe 	bl	0 <GRAPH_WhiteBlack>
  ea:	1cec      	adds	r4, r5, #3
C:\Documents and Settings\jarek\Pulpit\Privet\Magisterka\Programy\1\um0427\FWLib\project/SCROLL_M.c:71
  ec:	4621      	mov	r1, r4
  ee:	2002      	movs	r0, #2
  f0:	f7ff fffe 	bl	0 <GRAPH_TextGoTo>
C:\Documents and Settings\jarek\Pulpit\Privet\Magisterka\Programy\1\um0427\FWLib\project/SCROLL_M.c:72
  f4:	480c      	ldr	r0, [pc, #48]	(34 <printf+0x34>)
  f6:	f7ff fffe 	bl	0 <printf>
C:\Documents and Settings\jarek\Pulpit\Privet\Magisterka\Programy\1\um0427\FWLib\project/SCROLL_M.c:73
  fa:	4621      	mov	r1, r4
  fc:	2002      	movs	r0, #2
  fe:	f7ff fffe 	bl	0 <GRAPH_TextGoTo>
C:\Documents and Settings\jarek\Pulpit\Privet\Magisterka\Programy\1\um0427\FWLib\project/SCROLL_M.c:74
 102:	205b      	movs	r0, #91
 104:	f7ff fffe 	bl	0 <GRAPH_WriteChar>
C:\Documents and Settings\jarek\Pulpit\Privet\Magisterka\Programy\1\um0427\FWLib\project/SCROLL_M.c:75
 108:	6970      	ldr	r0, [r6, #20]
 10a:	f7ff fffe 	bl	0 <printf>
C:\Documents and Settings\jarek\Pulpit\Privet\Magisterka\Programy\1\um0427\FWLib\project/SCROLL_M.c:76
 10e:	205d      	movs	r0, #93
 110:	f7ff fffe 	bl	0 <GRAPH_WriteChar>
C:\Documents and Settings\jarek\Pulpit\Privet\Magisterka\Programy\1\um0427\FWLib\project/SCROLL_M.c:65
 114:	3501      	adds	r5, #1
 116:	3604      	adds	r6, #4
 118:	4a02      	ldr	r2, [pc, #8]	(124 <GoBack+0x124>)
 11a:	f992 303c 	ldrsb.w	r3, [r2, #60]
 11e:	429d      	cmp	r5, r3
 120:	dbdb      	blt.n	da <GoBack+0xda>
C:\Documents and Settings\jarek\Pulpit\Privet\Magisterka\Programy\1\um0427\FWLib\project/SCROLL_M.c:80
 122:	bd7c      	pop	{r2, r3, r4, r5, r6, pc}
	...
 12c:	00000024 	.word	0x00000024
Disassembly of section .text.Show:

00000000 <Show>:
Show():
C:\Documents and Settings\jarek\Pulpit\Privet\Magisterka\Programy\1\um0427\FWLib\project/SCROLL_M.c:110
   0:	4b77      	ldr	r3, [pc, #476]	(1e0 <Show+0x1e0>)
C:\Documents and Settings\jarek\Pulpit\Privet\Magisterka\Programy\1\um0427\FWLib\project/SCROLL_M.c:107
   2:	b570      	push	{r4, r5, r6, lr}
C:\Documents and Settings\jarek\Pulpit\Privet\Magisterka\Programy\1\um0427\FWLib\project/SCROLL_M.c:110
   4:	781b      	ldrb	r3, [r3, #0]
   6:	3b01      	subs	r3, #1
   8:	2b05      	cmp	r3, #5
   a:	f200 80e7 	bhi.w	1dc <Show+0x1dc>
   e:	e8df f003 	tbb	[pc, r3]
  12:	4003      	.short	0x4003
  14:	bbb97855 	.word	0xbbb97855
C:\Documents and Settings\jarek\Pulpit\Privet\Magisterka\Programy\1\um0427\FWLib\project/SCROLL_M.c:115
  18:	2101      	movs	r1, #1
  1a:	2002      	movs	r0, #2
  1c:	f7ff fffe 	bl	0 <GRAPH_TextGoTo>
C:\Documents and Settings\jarek\Pulpit\Privet\Magisterka\Programy\1\um0427\FWLib\project/SCROLL_M.c:116
  20:	f7ff fffe 	bl	0 <GRAPH_WhiteBlack>
C:\Documents and Settings\jarek\Pulpit\Privet\Magisterka\Programy\1\um0427\FWLib\project/SCROLL_M.c:117
  24:	486f      	ldr	r0, [pc, #444]	(1c0 <printf+0x1c0>)
  26:	f7ff fffe 	bl	0 <printf>
C:\Documents and Settings\jarek\Pulpit\Privet\Magisterka\Programy\1\um0427\FWLib\project/SCROLL_M.c:118
  2a:	2002      	movs	r0, #2
  2c:	2101      	movs	r1, #1
  2e:	f7ff fffe 	bl	0 <GRAPH_TextGoTo>
  32:	2400      	movs	r4, #0
C:\Documents and Settings\jarek\Pulpit\Privet\Magisterka\Programy\1\um0427\FWLib\project/SCROLL_M.c:119
  34:	e007      	b.n	46 <Show+0x46>
C:\Documents and Settings\jarek\Pulpit\Privet\Magisterka\Programy\1\um0427\FWLib\project/SCROLL_M.c:120
  36:	f852 0024 	ldr.w	r0, [r2, r4, lsl #2]
  3a:	f7ff fffe 	bl	0 <printf>
C:\Documents and Settings\jarek\Pulpit\Privet\Magisterka\Programy\1\um0427\FWLib\project/SCROLL_M.c:121
  3e:	486a      	ldr	r0, [pc, #424]	(1ac <printf+0x1ac>)
  40:	f7ff fffe 	bl	0 <printf>
C:\Documents and Settings\jarek\Pulpit\Privet\Magisterka\Programy\1\um0427\FWLib\project/SCROLL_M.c:119
  44:	3401      	adds	r4, #1
  46:	4a69      	ldr	r2, [pc, #420]	(1ec <Show+0x1ec>)
  48:	6d93      	ldr	r3, [r2, #88]
  4a:	429c      	cmp	r4, r3
  4c:	ddf3      	ble.n	36 <Show+0x36>
  4e:	f102 0614 	add.w	r6, r2, #20	; 0x14
  52:	2500      	movs	r5, #0
  54:	e016      	b.n	84 <Show+0x84>
  56:	1cec      	adds	r4, r5, #3
C:\Documents and Settings\jarek\Pulpit\Privet\Magisterka\Programy\1\um0427\FWLib\project/SCROLL_M.c:143
  58:	4621      	mov	r1, r4
  5a:	2002      	movs	r0, #2
  5c:	f7ff fffe 	bl	0 <GRAPH_TextGoTo>
C:\Documents and Settings\jarek\Pulpit\Privet\Magisterka\Programy\1\um0427\FWLib\project/SCROLL_M.c:144
  60:	4860      	ldr	r0, [pc, #384]	(184 <printf+0x184>)
  62:	f7ff fffe 	bl	0 <printf>
C:\Documents and Settings\jarek\Pulpit\Privet\Magisterka\Programy\1\um0427\FWLib\project/SCROLL_M.c:146
  66:	4621      	mov	r1, r4
  68:	2002      	movs	r0, #2
  6a:	f7ff fffe 	bl	0 <GRAPH_TextGoTo>
C:\Documents and Settings\jarek\Pulpit\Privet\Magisterka\Programy\1\um0427\FWLib\project/SCROLL_M.c:147
  6e:	205b      	movs	r0, #91
  70:	f7ff fffe 	bl	0 <GRAPH_WriteChar>
C:\Documents and Settings\jarek\Pulpit\Privet\Magisterka\Programy\1\um0427\FWLib\project/SCROLL_M.c:148
  74:	f856 0c04 	ldr.w	r0, [r6, #-4]
  78:	f7ff fffe 	bl	0 <printf>
C:\Documents and Settings\jarek\Pulpit\Privet\Magisterka\Programy\1\um0427\FWLib\project/SCROLL_M.c:149
  7c:	205d      	movs	r0, #93
  7e:	f7ff fffe 	bl	0 <GRAPH_WriteChar>
C:\Documents and Settings\jarek\Pulpit\Privet\Magisterka\Programy\1\um0427\FWLib\project/SCROLL_M.c:141
  82:	3501      	adds	r5, #1
  84:	4c59      	ldr	r4, [pc, #356]	(1ec <Show+0x1ec>)
  86:	3604      	adds	r6, #4
  88:	f994 303c 	ldrsb.w	r3, [r4, #60]
  8c:	429d      	cmp	r5, r3
  8e:	dbe2      	blt.n	56 <Show+0x56>
  90:	e05c      	b.n	14c <Show+0x14c>
C:\Documents and Settings\jarek\Pulpit\Privet\Magisterka\Programy\1\um0427\FWLib\project/SCROLL_M.c:165
  92:	f7ff fffe 	bl	0 <KEY_CheckKey>
  96:	f5b0 7f80 	cmp.w	r0, #256	; 0x100
  9a:	d007      	beq.n	ac <Show+0xac>
  9c:	f5b0 5f80 	cmp.w	r0, #4096	; 0x1000
  a0:	d002      	beq.n	a8 <Show+0xa8>
  a2:	2801      	cmp	r0, #1
  a4:	d004      	beq.n	b0 <Show+0xb0>
  a6:	e099      	b.n	1dc <Show+0x1dc>
C:\Documents and Settings\jarek\Pulpit\Privet\Magisterka\Programy\1\um0427\FWLib\project/SCROLL_M.c:167
  a8:	2203      	movs	r2, #3
  aa:	e002      	b.n	b2 <Show+0xb2>
C:\Documents and Settings\jarek\Pulpit\Privet\Magisterka\Programy\1\um0427\FWLib\project/SCROLL_M.c:171
  ac:	2204      	movs	r2, #4
  ae:	e000      	b.n	b2 <Show+0xb2>
C:\Documents and Settings\jarek\Pulpit\Privet\Magisterka\Programy\1\um0427\FWLib\project/SCROLL_M.c:175
  b0:	2206      	movs	r2, #6
  b2:	4b4b      	ldr	r3, [pc, #300]	(1e0 <Show+0x1e0>)
  b4:	701a      	strb	r2, [r3, #0]
C:\Documents and Settings\jarek\Pulpit\Privet\Magisterka\Programy\1\um0427\FWLib\project/SCROLL_M.c:176
  b6:	f7ff fffe 	bl	0 <KEY_KeyServed>
  ba:	e08f      	b.n	1dc <Show+0x1dc>
C:\Documents and Settings\jarek\Pulpit\Privet\Magisterka\Programy\1\um0427\FWLib\project/SCROLL_M.c:181
  bc:	4c4b      	ldr	r4, [pc, #300]	(1ec <Show+0x1ec>)
  be:	6c63      	ldr	r3, [r4, #68]
  c0:	2b00      	cmp	r3, #0
  c2:	f000 8088 	beq.w	1d6 <Show+0x1d6>
C:\Documents and Settings\jarek\Pulpit\Privet\Magisterka\Programy\1\um0427\FWLib\project/SCROLL_M.c:182
  c6:	f7ff fffe 	bl	0 <GRAPH_WhiteBlack>
C:\Documents and Settings\jarek\Pulpit\Privet\Magisterka\Programy\1\um0427\FWLib\project/SCROLL_M.c:183
  ca:	6c61      	ldr	r1, [r4, #68]
  cc:	2002      	movs	r0, #2
  ce:	3103      	adds	r1, #3
  d0:	f7ff fffe 	bl	0 <GRAPH_TextGoTo>
C:\Documents and Settings\jarek\Pulpit\Privet\Magisterka\Programy\1\um0427\FWLib\project/SCROLL_M.c:184
  d4:	4843      	ldr	r0, [pc, #268]	(110 <printf+0x110>)
  d6:	f7ff fffe 	bl	0 <printf>
C:\Documents and Settings\jarek\Pulpit\Privet\Magisterka\Programy\1\um0427\FWLib\project/SCROLL_M.c:185
  da:	6c61      	ldr	r1, [r4, #68]
  dc:	2002      	movs	r0, #2
  de:	3103      	adds	r1, #3
  e0:	f7ff fffe 	bl	0 <GRAPH_TextGoTo>
C:\Documents and Settings\jarek\Pulpit\Privet\Magisterka\Programy\1\um0427\FWLib\project/SCROLL_M.c:186
  e4:	205b      	movs	r0, #91
  e6:	f7ff fffe 	bl	0 <GRAPH_WriteChar>
C:\Documents and Settings\jarek\Pulpit\Privet\Magisterka\Programy\1\um0427\FWLib\project/SCROLL_M.c:187
  ea:	6c63      	ldr	r3, [r4, #68]
  ec:	eb04 0383 	add.w	r3, r4, r3, lsl #2
  f0:	6958      	ldr	r0, [r3, #20]
  f2:	f7ff fffe 	bl	0 <printf>
C:\Documents and Settings\jarek\Pulpit\Privet\Magisterka\Programy\1\um0427\FWLib\project/SCROLL_M.c:188
  f6:	205d      	movs	r0, #93
  f8:	f7ff fffe 	bl	0 <GRAPH_WriteChar>
C:\Documents and Settings\jarek\Pulpit\Privet\Magisterka\Programy\1\um0427\FWLib\project/SCROLL_M.c:189
  fc:	6c63      	ldr	r3, [r4, #68]
  fe:	3b01      	subs	r3, #1
 100:	e023      	b.n	14a <Show+0x14a>
C:\Documents and Settings\jarek\Pulpit\Privet\Magisterka\Programy\1\um0427\FWLib\project/SCROLL_M.c:201
 102:	4c3a      	ldr	r4, [pc, #232]	(1ec <Show+0x1ec>)
 104:	f994 303c 	ldrsb.w	r3, [r4, #60]
 108:	6c62      	ldr	r2, [r4, #68]
 10a:	3b01      	subs	r3, #1
 10c:	429a      	cmp	r2, r3
 10e:	d062      	beq.n	1d6 <Show+0x1d6>
C:\Documents and Settings\jarek\Pulpit\Privet\Magisterka\Programy\1\um0427\FWLib\project/SCROLL_M.c:202
 110:	f7ff fffe 	bl	0 <GRAPH_WhiteBlack>
C:\Documents and Settings\jarek\Pulpit\Privet\Magisterka\Programy\1\um0427\FWLib\project/SCROLL_M.c:203
 114:	6c61      	ldr	r1, [r4, #68]
 116:	2002      	movs	r0, #2
 118:	3103      	adds	r1, #3
 11a:	f7ff fffe 	bl	0 <GRAPH_TextGoTo>
C:\Documents and Settings\jarek\Pulpit\Privet\Magisterka\Programy\1\um0427\FWLib\project/SCROLL_M.c:204
 11e:	4831      	ldr	r0, [pc, #196]	(c8 <printf+0xc8>)
 120:	f7ff fffe 	bl	0 <printf>
C:\Documents and Settings\jarek\Pulpit\Privet\Magisterka\Programy\1\um0427\FWLib\project/SCROLL_M.c:205
 124:	6c61      	ldr	r1, [r4, #68]
 126:	2002      	movs	r0, #2
 128:	3103      	adds	r1, #3
 12a:	f7ff fffe 	bl	0 <GRAPH_TextGoTo>
C:\Documents and Settings\jarek\Pulpit\Privet\Magisterka\Programy\1\um0427\FWLib\project/SCROLL_M.c:206
 12e:	205b      	movs	r0, #91
 130:	f7ff fffe 	bl	0 <GRAPH_WriteChar>
C:\Documents and Settings\jarek\Pulpit\Privet\Magisterka\Programy\1\um0427\FWLib\project/SCROLL_M.c:207
 134:	6c63      	ldr	r3, [r4, #68]
 136:	eb04 0383 	add.w	r3, r4, r3, lsl #2
 13a:	6958      	ldr	r0, [r3, #20]
 13c:	f7ff fffe 	bl	0 <printf>
C:\Documents and Settings\jarek\Pulpit\Privet\Magisterka\Programy\1\um0427\FWLib\project/SCROLL_M.c:208
 140:	205d      	movs	r0, #93
 142:	f7ff fffe 	bl	0 <GRAPH_WriteChar>
C:\Documents and Settings\jarek\Pulpit\Privet\Magisterka\Programy\1\um0427\FWLib\project/SCROLL_M.c:209
 146:	6c63      	ldr	r3, [r4, #68]
 148:	3301      	adds	r3, #1
 14a:	6463      	str	r3, [r4, #68]
C:\Documents and Settings\jarek\Pulpit\Privet\Magisterka\Programy\1\um0427\FWLib\project/SCROLL_M.c:210
 14c:	f7ff fffe 	bl	0 <GRAPH_BlackWhite>
C:\Documents and Settings\jarek\Pulpit\Privet\Magisterka\Programy\1\um0427\FWLib\project/SCROLL_M.c:211
 150:	6c61      	ldr	r1, [r4, #68]
 152:	2002      	movs	r0, #2
 154:	3103      	adds	r1, #3
 156:	f7ff fffe 	bl	0 <GRAPH_TextGoTo>
C:\Documents and Settings\jarek\Pulpit\Privet\Magisterka\Programy\1\um0427\FWLib\project/SCROLL_M.c:212
 15a:	4822      	ldr	r0, [pc, #136]	(8c <printf+0x8c>)
 15c:	f7ff fffe 	bl	0 <printf>
C:\Documents and Settings\jarek\Pulpit\Privet\Magisterka\Programy\1\um0427\FWLib\project/SCROLL_M.c:213
 160:	6c61      	ldr	r1, [r4, #68]
 162:	2002      	movs	r0, #2
 164:	3103      	adds	r1, #3
 166:	f7ff fffe 	bl	0 <GRAPH_TextGoTo>
C:\Documents and Settings\jarek\Pulpit\Privet\Magisterka\Programy\1\um0427\FWLib\project/SCROLL_M.c:214
 16a:	205b      	movs	r0, #91
 16c:	f7ff fffe 	bl	0 <GRAPH_WriteChar>
C:\Documents and Settings\jarek\Pulpit\Privet\Magisterka\Programy\1\um0427\FWLib\project/SCROLL_M.c:215
 170:	6c63      	ldr	r3, [r4, #68]
 172:	eb04 0383 	add.w	r3, r4, r3, lsl #2
 176:	6958      	ldr	r0, [r3, #20]
 178:	f7ff fffe 	bl	0 <printf>
C:\Documents and Settings\jarek\Pulpit\Privet\Magisterka\Programy\1\um0427\FWLib\project/SCROLL_M.c:216
 17c:	205d      	movs	r0, #93
 17e:	f7ff fffe 	bl	0 <GRAPH_WriteChar>
 182:	e028      	b.n	1d6 <Show+0x1d6>
C:\Documents and Settings\jarek\Pulpit\Privet\Magisterka\Programy\1\um0427\FWLib\project/SCROLL_M.c:222
 184:	2200      	movs	r2, #0
 186:	e027      	b.n	1d8 <Show+0x1d8>
C:\Documents and Settings\jarek\Pulpit\Privet\Magisterka\Programy\1\um0427\FWLib\project/SCROLL_M.c:226
 188:	4918      	ldr	r1, [pc, #96]	(1ec <Show+0x1ec>)
 18a:	6c4a      	ldr	r2, [r1, #68]
 18c:	6c0b      	ldr	r3, [r1, #64]
 18e:	eb01 0282 	add.w	r2, r1, r2, lsl #2
 192:	6a92      	ldr	r2, [r2, #40]
 194:	601a      	str	r2, [r3, #0]
C:\Documents and Settings\jarek\Pulpit\Privet\Magisterka\Programy\1\um0427\FWLib\project/SCROLL_M.c:228
 196:	6c48      	ldr	r0, [r1, #68]
 198:	b960      	cbnz	r0, 1b4 <Show+0x1b4>
C:\Documents and Settings\jarek\Pulpit\Privet\Magisterka\Programy\1\um0427\FWLib\project/SCROLL_M.c:229
 19a:	6c8b      	ldr	r3, [r1, #72]
 19c:	644b      	str	r3, [r1, #68]
C:\Documents and Settings\jarek\Pulpit\Privet\Magisterka\Programy\1\um0427\FWLib\project/SCROLL_M.c:230
 19e:	6ccb      	ldr	r3, [r1, #76]
 1a0:	648b      	str	r3, [r1, #72]
C:\Documents and Settings\jarek\Pulpit\Privet\Magisterka\Programy\1\um0427\FWLib\project/SCROLL_M.c:231
 1a2:	6d0b      	ldr	r3, [r1, #80]
 1a4:	64cb      	str	r3, [r1, #76]
C:\Documents and Settings\jarek\Pulpit\Privet\Magisterka\Programy\1\um0427\FWLib\project/SCROLL_M.c:232
 1a6:	6d4b      	ldr	r3, [r1, #84]
C:\Documents and Settings\jarek\Pulpit\Privet\Magisterka\Programy\1\um0427\FWLib\project/SCROLL_M.c:233
 1a8:	6548      	str	r0, [r1, #84]
C:\Documents and Settings\jarek\Pulpit\Privet\Magisterka\Programy\1\um0427\FWLib\project/SCROLL_M.c:232
 1aa:	650b      	str	r3, [r1, #80]
C:\Documents and Settings\jarek\Pulpit\Privet\Magisterka\Programy\1\um0427\FWLib\project/SCROLL_M.c:234
 1ac:	6d8b      	ldr	r3, [r1, #88]
 1ae:	3b01      	subs	r3, #1
 1b0:	658b      	str	r3, [r1, #88]
 1b2:	e010      	b.n	1d6 <Show+0x1d6>
C:\Documents and Settings\jarek\Pulpit\Privet\Magisterka\Programy\1\um0427\FWLib\project/SCROLL_M.c:237
 1b4:	6d8b      	ldr	r3, [r1, #88]
C:\Documents and Settings\jarek\Pulpit\Privet\Magisterka\Programy\1\um0427\FWLib\project/SCROLL_M.c:238
 1b6:	eb01 0280 	add.w	r2, r1, r0, lsl #2
 1ba:	6952      	ldr	r2, [r2, #20]
C:\Documents and Settings\jarek\Pulpit\Privet\Magisterka\Programy\1\um0427\FWLib\project/SCROLL_M.c:237
 1bc:	3301      	adds	r3, #1
 1be:	658b      	str	r3, [r1, #88]
C:\Documents and Settings\jarek\Pulpit\Privet\Magisterka\Programy\1\um0427\FWLib\project/SCROLL_M.c:238
 1c0:	f841 2023 	str.w	r2, [r1, r3, lsl #2]
C:\Documents and Settings\jarek\Pulpit\Privet\Magisterka\Programy\1\um0427\FWLib\project/SCROLL_M.c:239
 1c4:	6d0b      	ldr	r3, [r1, #80]
 1c6:	654b      	str	r3, [r1, #84]
C:\Documents and Settings\jarek\Pulpit\Privet\Magisterka\Programy\1\um0427\FWLib\project/SCROLL_M.c:240
 1c8:	6ccb      	ldr	r3, [r1, #76]
 1ca:	650b      	str	r3, [r1, #80]
C:\Documents and Settings\jarek\Pulpit\Privet\Magisterka\Programy\1\um0427\FWLib\project/SCROLL_M.c:241
 1cc:	6c8b      	ldr	r3, [r1, #72]
C:\Documents and Settings\jarek\Pulpit\Privet\Magisterka\Programy\1\um0427\FWLib\project/SCROLL_M.c:242
 1ce:	6488      	str	r0, [r1, #72]
C:\Documents and Settings\jarek\Pulpit\Privet\Magisterka\Programy\1\um0427\FWLib\project/SCROLL_M.c:241
 1d0:	64cb      	str	r3, [r1, #76]
C:\Documents and Settings\jarek\Pulpit\Privet\Magisterka\Programy\1\um0427\FWLib\project/SCROLL_M.c:243
 1d2:	2300      	movs	r3, #0
 1d4:	644b      	str	r3, [r1, #68]
C:\Documents and Settings\jarek\Pulpit\Privet\Magisterka\Programy\1\um0427\FWLib\project/SCROLL_M.c:245
 1d6:	2202      	movs	r2, #2
 1d8:	4b01      	ldr	r3, [pc, #4]	(1e0 <Show+0x1e0>)
 1da:	701a      	strb	r2, [r3, #0]
C:\Documents and Settings\jarek\Pulpit\Privet\Magisterka\Programy\1\um0427\FWLib\project/SCROLL_M.c:248
 1dc:	bd70      	pop	{r4, r5, r6, pc}
 1de:	46c0      	nop			(mov r8, r8)
	...
 1e8:	00000024 	.word	0x00000024
 1ec:	00000000 	.word	0x00000000
